:1000000028C04CC042C24AC049C0F5C147C046C022
:1000100045C044C043C042C041C040C03FC00000D2
:10002000000036000000000037000000000038002B
:10003000020202020202020202020102040810206D
:1000400020041008010200000400000000007103F9
:10005000DA0311241FBECFE5D1E0DEBFCDBF10E033
:10006000A0E6B0E0EEE5F8E002C005900D92A83CF5
:10007000B107D9F721E0A8ECB0E001C01D92A4338C
:10008000B207E1F710E0C8E2D0E003C02197FE011B
:10009000D4D3C732D107D1F770D2D5C3B1CF089529
:1000A000AF92BF92CF92DF92EF92FF920F931F9386
:1000B000CF93DF936C017B018B01040F151FEB01C4
:1000C0005E01AE18BF08C017D10759F06991D6017B
:1000D000ED91FC910190F081E02DC6010995892BED
:1000E00079F7C501DF91CF911F910F91FF90EF90AC
:1000F000DF90CF90BF90AF90089590E0FC01EC5B53
:10010000FF4F3491FC01E65CFF4F2491FC01E05D60
:10011000FF4FE491EE23B9F0332329F0323001F19F
:1001200098F43130C9F0F0E0EE0FFF1FE65DFF4FAD
:10013000A591B4918FB7F894EC91611114C02095FA
:100140002E232C938FBF0895333011F0343059F79C
:100150008CB58F7D8CBDE7CF8AB58F778ABDE3CF15
:100160008AB58F7DFBCF2E2BECCFCF93DF9390E022
:10017000FC01E65CFF4F2491805D9F4FFC01849160
:100180008823D1F090E0880F991FFC01EC5DFF4FB0
:10019000A591B491FC01E65DFF4FC591D491611129
:1001A0000EC09FB7F8948C91E22FE0958E238C932C
:1001B0002881E223E8839FBFDF91CF9108958FB715
:1001C000F894EC91E22BEC938FBFF6CF3FB7F89405
:1001D00080910D0190910E01A0910F01B09110013D
:1001E00022B708B601FE05C02F3F19F00196A11DE8
:1001F000B11D3FBFBA2FA92F982F8827BC01CD0171
:10020000620F711D811D911D43E0660F771F881FCE
:10021000991F4A95D1F708958F929F92AF92BF92FE
:10022000CF92DF92EF92FF92D1DF4B015C0180ED24
:10023000C82E87E0D82EE12CF12CC8DF6819790987
:100240008A099B09683E734081059105B0F321E05E
:10025000C21AD108E108F10888EE880E83E0981EE2
:10026000A11CB11CC114D104E104F10431F7FF90C9
:10027000EF90DF90CF90BF90AF909F908F900895B8
:1002800020911301309114012817390771F49091CE
:10029000110180911201981741F0E0911101F0E0F5
:1002A000E853FF4F808190E008958FEF9FEF08950E
:1002B000EF92FF920F931F93CF93DF93DC015C9635
:1002C000ED90FC905D97E114F10479F481E090E009
:1002D00013969C938E93129790E080E0DF91CF91DC
:1002E0001F910F91FF90EF9008955196ED91FC9121
:1002F000529750968C915097982F90950FB75E9685
:100300002C915E97122F127021FD6095F894208138
:10031000112319F1282B2083E7012197F1F728E019
:10032000462F50E0308160FF1AC0382B3083E70140
:100330002197F1F7BA0175956795215089F7112337
:1003400081F08081892380830FBF5C968D919C9181
:100350000197F1F781E090E0C1CF2923DCCF392369
:10036000E5CF9081892BEFCF2091130130911401BB
:100370002817390769F4809112012091110190E04A
:10038000805C9F4F821B910960E470E02FD208953A
:1003900090E080E008952091130130911401281716
:1003A0003907B9F49091110180911201981789F0E1
:1003B000E0911101F0E0E853FF4F8081209111019D
:1003C00030E02F5F3F4F2F7333272093110190E0D0
:1003D00008958FEF9FEF089590E080E00895FC016D
:1003E00001900020E9F73197AF01481B590BBC0180
:1003F00085E191E055CE1F920F920FB60F92112416
:100400002F933F938F939F93AF93BF938091090155
:1004100090910A01A0910B01B0910C01309108015B
:1004200026E0230F2D3758F50296A11DB11D20930C
:1004300008018093090190930A01A0930B01B093E6
:100440000C0180910D0190910E01A0910F01B091CE
:1004500010010196A11DB11D80930D0190930E0115
:10046000A0930F01B0931001BF91AF919F918F9115
:100470003F912F910F900FBE0F901F90189529E874
:10048000230F0396A11DB11DD2CF1F920F920FB65D
:100490000F9211242F933F934F935F936F937F930A
:1004A0008F939F93AF93BF93EF93FF93E0911301CB
:1004B000F0911401309749F0A685B7858585968D12
:1004C00091FF14C09C918923A1F4FF91EF91BF91FA
:1004D000AF919F918F917F916F915F914F913F91DC
:1004E0002F910F900FBE0F901F9018959C9189230C
:1004F00061F7A389B4899C918589809589238C9320
:10050000868997890197F1F7608D718DA685B785EA
:10051000558538E020E0CB010197F1F7822F90E07C
:1005200095958795282F4C91452309F020683150E7
:1005300091F7868D81FD20958091120190E00196C2
:100540008F73992730911101381799F0A0911201FA
:10055000B0E0A853BF4F2C9380931201828D938DEE
:100560000197F1F7A389B4898C919589892B8C9394
:10057000ACCF868D8160868FF1CF78948AB582600A
:100580008ABD8AB581608ABD83B7826083BF83B725
:10059000816083BF89B7826089BF80B7826080BF76
:1005A00080B7816080BF329A319A3098379A8CB583
:1005B00080648CBD60E082E0D8DD61E083E0D5DD61
:1005C0001092300110922F0110922E0110922D01E5
:1005D00010922C0110922B018DEC90E0909332013F
:1005E0008093310130912101353020F545E550E00F
:1005F00050932C0140932B014BEC50E050932E0173
:1006000040932D0140E950E05093300140932F0179
:100610002BB720622BBF45E350E050932901409354
:10062000280121E001C0220F3A95EAF720932A0120
:100630000197F1F780912F0190913001892B49F1B9
:10064000E0911301F091140181E0E531F80709F11F
:10065000309739F0A389B4899C9185898095892345
:100660008C93809133018E7F80933301109212011D
:100670001092110185E191E0909314018093130190
:10068000E0912801F0912901808190912A01892B24
:10069000808382E790E0A3DE80E890E0A0DE85E939
:1006A00090E09DDE83EA90E09ADEB6DD81EB90E09B
:1006B00096DEB2DD61E084E058DD61E084E01DDDBE
:1006C000D0E0C0E085E191E04FDE892BD9F385E1F0
:1006D00091E061DE219661E0C0FD60E084E00DDD27
:1006E000F1CF109218011092170188EE93E0A0E06C
:1006F000B0E08093190190931A01A0931B01B0936D
:100700001C0184E690E090931601809315011092ED
:100710002C0110922B0110922E0110922D0110929B
:10072000300110922F01109232011092310160912C
:1007300033016E7F6D7F609333016695617081E058
:10074000682783E0DADC61E083E00FDDEDE3F0E0D1
:10075000E491E0932501E3E3F0E0E491F0E0EE0FB3
:10076000FF1FE65DFF4F8591949190932701809341
:10077000260160E082E0F9DC8091330181FD03C055
:1007800061E082E0BADC82E080932101ECE3F0E0FA
:10079000E491E0932201E2E3F0E0E491F0E0EE0F77
:1007A000FF1FE25EFF4F8591949190932401809307
:1007B0002301089584E690E090931601809315013B
:1007C00080911301909114018551914071F4E09151
:1007D0002801F0912901908180912A018095892337
:1007E00080831092140110921301089597FB072E35
:1007F00016F4009406D077FD08D00BD007FC05D086
:100800003EF4909581959F4F0895709561957F4F27
:100810000895AA1BBB1B51E107C0AA1FBB1FA61747
:10082000B70710F0A61BB70B881F991F5A95A9F799
:1008300080959095BC01CD010895EE0FFF1F0590A6
:10084000F491E02D099410E0C8E2D0E003C0FE016D
:0E085000F4DF2196C932D107D1F7F894FFCF1B
:10085E000000000058015000EC014F00B401CB0124
:10086E0040010D0A2B5354574D4F443D300D0A0095
:10087E000D0A2B53544E413D4D616B6572626C6F88
:10088E00636B0D0A000D0A2B53544F4155543D31E5
:10089E000D0A000D0A2B53544155544F3D300D0A8D
:1008AE0000626C7565746F6F746820636F6E6E6531
:0808BE0063746564210A000067
:00000001FF
